:1000000019C033C032C031C030C02FC02EC02DC087
:100010002CC02BC058C029C028C028C026C025C06D
:1000200024C023C022C021C020C01FC01EC01DC0CC
:100030001CC01BC011241FBEC0E0D4E0DEBFCDBF7A
:1000400011E0A0E0B1E0E4EEFBE002C005900D920B
:10005000A633B107D9F711E0A6E3B1E001C01D92C4
:10006000A736B107E1F77DD2BBC5CACF1F920F9269
:100070000FB60F9211248F939F93809160019091FE
:100080006101019690936101809360017894809161
:10009000400190914101019690934101809340016C
:1000A00080915701882339F08091570181508093C6
:1000B00057015D9A01C05D989F918F910F900FBE7F
:1000C0000F901F9018951F920F920FB60F92112448
:1000D0002F938F939F93AF93BF938091370190910C
:1000E0003801A0913901B0913A010196A11DB11DCD
:1000F0008093370190933801A0933901B0933A016E
:1001000020916601213061F5809352019093530153
:10011000A0935401B093550180918600909187007F
:1001200090935D0180935C018091600190916101E9
:1001300090935F0180935E01B09B0FC080915C0142
:1001400090915D0197FD09C080915E0190915F01E2
:10015000019690935F0180935E0182E08093660137
:10016000BF91AF919F918F912F910F900FBE0F90E4
:100170001F901895F999FECF92BD81BDF89A80B570
:100180000895F999FECF72BD61BDF89A90B58917AF
:1001900041F0F89472BD61BD80BD84E08FBBF99AD7
:1001A000789408950F931F93DF93CF930F92CDB759
:1001B000DEB78B019983E5DFB8016F5F7F4F9981CF
:1001C000892FDFDF0F90CF91DF911F910F9108955D
:1001D000F999FECF92BD81BDF89A40B5F999FECF4D
:1001E000019692BD81BDF89A80B5382F20E0240F8A
:1001F000311DC9010895DF93CF930F92CDB7DEB7BC
:1002000082E3898306C081EE94E00197F1F700C094
:1002100000008981982F915099838823A1F70F902E
:10022000CF91DF910895419A84E08A95F1F700001B
:100230004198089595B1869586958C73937C892B0A
:1002400085B9F1DF0895F6DF83ED90E30197F1F7CB
:1002500000C0000008951F93182F662311F0409AE4
:1002600001C04098812FE6DF812F8295807FE2DFF9
:1002700081EE94E00197F1F700C000001F9108950E
:1002800061E0E9DF0895CF93DF93EC0101C0F8DF6F
:1002900089918823E1F7DF91CF910895AF92BF92C2
:1002A000CF92DF92EF92FF920F931F937B018C010D
:1002B000D42E2FE632E143E85AE32BD487FF07C060
:1002C00012E000E0FF24EE24DD24CC248EC0DD20EB
:1002D00059F4C801B70120E030E040E752E41DD4F2
:1002E0006B017C0112E017C060E070E080E89FE3E2
:1002F000A8019701C3D26B017C0114E00CC06C2DE6
:100300007D2D8E2D9F2D20E030E04AE754E405D46A
:100310006B017C011F5F6C2D7D2D8E2D9F2D20E0AC
:1003200030E040E85FE3A6D287FDE9CF0CC06C2D3A
:100330007D2D8E2D9F2D2FE632E143E85AE3EDD33C
:100340006B017C0111506C2D7D2D8E2D9F2D20E099
:1003500030E04AE754E4DDD387FFE9CF00E00CC08A
:100360006C2D7D2D8E2D9F2D2DEC3CEC4CEC5DE30A
:10037000D4D36B017C010F5F6C2D7D2D8E2D9F2DB5
:1003800020E030E040E251E4C4D387FFE9CF6C2D98
:100390007D2D8E2D9F2D2CEA35EC47EA56E306D2B3
:1003A000F62EE72ED82EC92EA7019601652F742FA1
:1003B000832F922F20E030E040E251E4AAD388233B
:1003C000A4F0A7019601652F742F832F922F2DEC97
:1003D0003CEC4CEC5DE3A1D3F62EE72ED82EC92ED3
:1003E0000F5F033014F0115000E0BB24A701960109
:1003F000652F7E2D832F9C2DA9D2A62E862F805D62
:100400003FDFB01611F48EE23BDFB39486E0B816FE
:10041000D1F06A2D772767FD7095872F972FC9D266
:100420009B01AC01D701F6016B2F7E2D8F2F9C2DE8
:10043000BCD120E030E040E251E46FD3F62EE72E4D
:10044000D82EC92ED3CF80E21BDF85E01802C00171
:1004500011248E5E9E4F17DF80E212DF1F910F91F5
:10046000FF90EF90DF90CF90BF90AF90089560E045
:10047000F2DE0895CF92DF92EF92FF921F93CF9317
:10048000DF9316B110951470809136018095812309
:1004900009F442C0C0903B01D0903C01E0903D0186
:1004A000F0903E01C701B60127E73EEB4FE75FE35F
:1004B00030D318168CF5C701B60125EC30E240E8C0
:1004C0005FE3D8D1882344F5809162019091630164
:1004D000A0916401B0916501EC01C050DD42BE0104
:1004E000882777FD8095982F6050734D8E4C9E4FD6
:1004F00060D260934E0170934F01809350019093AE
:10050000510184E8B4DF80E091E0BDDECE0162E01D
:1005100070E048DE1092560110933601DF91CF91C2
:100520001F91FF90EF90DF90CF90089564DE80E3FD
:100530008ADE80E388DE80E386DE80E284DE88E295
:1005400096DF8CE094DF81E092DF55DE80E88FDF7C
:100550008CE091E098DE80EC8ADF8FE091E093DE22
:1005600008958F929F92AF92BF92CF92DF92EF92B7
:10057000FF920F931F9380E88093610010926100B7
:1005800083E085B99CE398B92FE12BB994B987B979
:1005900080E28AB9CBDF1092560180B7846080BFB9
:1005A0001092660181E08093810081E280936F0068
:1005B00082E090E00DDE9C01B901882777FD8095EF
:1005C000982F6050734D8E4C9E4FF3D160934E0127
:1005D00070934F018093500190935101789411E0F2
:1005E0000EE180916F008E7F80936F008091660195
:1005F000882369F4809140019091410184369105EE
:1006000030F01093660110924101109240018091E8
:100610006F00816080936F0080916601823009F7DE
:1006200080915E0190915F0120915C0130915D01AC
:10063000A0E0B0E0DC019927882740E050E0820F7D
:10064000931FA41FB51F8093580190935901A09345
:100650005A01B0935B018091580190915901A0918A
:100660005A01B0915B0120914201309143014091C8
:10067000440150914501821B930BA40BB50B809351
:10068000620190936301A0936401B093650180912E
:10069000580190915901A0915A01B0915B0180934A
:1006A000420190934301A0934401B093450180918E
:1006B000520190915301A0915401B09155012091A4
:1006C0004601309147014091480150914901821BF8
:1006D000930BA40BB50B80934A0190934B01A0930D
:1006E0004C01B0934D018091520190915301A09122
:1006F0005401B09155018093460190934701A09316
:100700004801B093490110926601809156018823F7
:1007100009F448C00093570160914A0170914B0160
:1007200080914C0190914D01C0906201D090630185
:10073000E0906401F09065013AD120914E01309132
:100740004F014091500150915101E7D14B015C01A3
:10075000C701B6012CD19B01AC01C501B4018ED0FB
:1007600060933B0170933C0180933D0190933E0167
:1007700084E87DDE60913B0170913C0180913D01F8
:1007800090913E0140E08ADD84EC71DE60913B0196
:1007900070913C0180913D0190913E0141E07EDDF0
:1007A00069DE1FCF109356011CCF5058BB27AA27D4
:1007B0000ED075C166D130F06BD120F031F49F3F7F
:1007C00011F41EF45BC10EF4E095E7FB51C1E92F73
:1007D00077D180F3BA17620773078407950718F07B
:1007E00071F49EF58FC10EF4E0950B2EBA2FA02D5B
:1007F0000B01B90190010C01CA01A0011124FF27CE
:10080000591B99F0593F50F4503E68F11A16F040C8
:10081000A22F232F342F4427585FF3CF46953795C7
:100820002795A795F0405395C9F77EF41F16BA0B8C
:10083000620B730B840BBAF09150A1F0FF0FBB1F3A
:10084000661F771F881FC2F70EC0BA0F621F731F83
:10085000841F48F4879577956795B795F7959E3FE0
:1008600008F0B3CF9395880F08F09927EE0F97956E
:1008700087950895D9D008F481E008950CD00FC170
:1008800007D140F0FED030F021F45F3F19F0F0C006
:10089000511139C1F3C014D198F39923C9F35523E9
:1008A000B1F3951B550BBB27AA2762177307840763
:1008B00038F09F5F5F4F220F331F441FAA1FA9F319
:1008C00033D00E2E3AF0E0E830D091505040E6950B
:1008D000001CCAF729D0FE2F27D0660F771F881F6C
:1008E000BB1F261737074807AB07B0E809F0BB0B5B
:1008F000802DBF01FF2793585F4F2AF09E3F51057F
:1009000068F0B6C000C15F3FECF3983EDCF386951B
:1009100077956795B795F7959F5FC9F7880F911DF4
:100920009695879597F90895E1E0660F771F881FE0
:10093000BB1F621773078407BA0720F0621B730B93
:10094000840BBA0BEE1F88F7E095089504D06894E5
:10095000B111D9C00895BCD088F09F5790F0B92F3D
:100960009927B751A0F0D1F0660F771F881F991F04
:100970001AF0BA95C9F712C0B13081F0C3D0B1E016
:100980000895C0C0672F782F8827B85F39F0B93F26
:10099000CCF3869577956795B395D9F73EF4909506
:1009A0008095709561957F4F8F4F9F4F0895E89484
:1009B00009C097FB3EF490958095709561957F4FA7
:1009C0008F4F9F4F9923A9F0F92F96E9BB27939555
:1009D000F695879577956795B795F111F8CFFAF465
:1009E000BB0F11F460FF1BC06F5F7F4F8F4F9F4F96
:1009F00016C0882311F096E911C0772321F09EE8F4
:100A0000872F762F05C0662371F096E8862F70E059
:100A100060E02AF09A95660F771F881FDAF7880F33
:100A20009695879597F90895990F0008550FAA0B89
:100A3000E0E8FEEF16161706E807F907C0F01216F1
:100A40001306E407F50798F0621B730B840B950BF4
:100A500039F40A2661F0232B242B252B21F4089549
:100A60000A2609F4A140A6958FEF811D811D0895E6
:100A700097F99F6780E870E060E008959FEF80EC51
:100A8000089500240A9416161706180609060895F4
:100A900000240A9412161306140605060895092E5A
:100AA0000394000C11F4882352F0BB0F40F4BF2BC9
:100AB00011F460FF04C06F5F7F4F8F4F9F4F089509
:100AC00057FD9058440F551F59F05F3F71F04795FF
:100AD000880F97FB991F61F09F3F79F087950895E4
:100AE000121613061406551FF2CF4695F1DF08C003
:100AF000161617061806991FF1CF86957105610520
:100B000008940895E894BB2766277727CB0197F9C7
:100B100008958ADF08F48FEF08950BD0C0CFB1DFBE
:100B200028F0B6DF18F0952309F0A2CFA7CF112443
:100B3000EACFC6DFA0F3959FD1F3950F50E0551F84
:100B4000629FF001729FBB27F00DB11D639FAA2722
:100B5000F00DB11DAA1F649F6627B00DA11D661F71
:100B6000829F2227B00DA11D621F739FB00DA11D92
:100B7000621F839FA00D611D221F749F3327A00D4C
:100B8000611D231F849F600D211D822F762F6A2FE8
:100B900011249F5750408AF0E1F088234AF0EE0F6D
:100BA000FF1FBB1F661F771F881F91505040A9F77A
:100BB0009E3F510570F05CCFA6CF5F3FECF3983EAF
:100BC000DCF3869577956795B795F795E7959F5FE1
:100BD000C1F7FE2B880F911D9695879597F908957B
:040BE000F894FFCFB7
:100BE4004B616C2E2046455254494700443A005408
:100BF4003A004D72706D006B72706D0072706D20F2
:100C0400006D72706D0073656B20006D73202000A1
:060C1400757320200000B2
:00000001FF
